:020000000528D1
:080008002E288316013085004B
:10001000880186018701831281309F0083160E308C
:100020009F0083129101FF3095018316FF309200EB
:100030008312063092000C3097008F018E01093038
:100040009C00C4309B00013090000B309D00831653
:1000500001308D008312C0308B002D288D011F19B7
:100060002F281E0886000609950086091509A0009C
:100070001030200203183E28453069282030200225
:1000800003184428403069284030200203184A28C9
:100090003530692860302002031850283030692834
:1000A000803020020318562825306928A03020020D
:1000B00003185C2820306928C03020020318622809
:1000C00015306928E03020020318682810306928AC
:0600D00000308800090069
:02400E00F23F7F
:00000001FF
